:1000000000308A00762800000A108A100A11820740
:1000100050346534723469346F346434613420345C
:10002000253435344C3475342034753473342E34DF
:100030000A340D340034AC010408AB002C10831BCF
:100040002C14250EF038A700A707E23EA800323E88
:10005000AA0025080F39A807A807AA07E93EA900A2
:10006000A907A907240E0F39A907AA07A90DAA0DE8
:10007000AA09AA0D24080F39AA07A70D0730A60060
:100080000A30AA07A903031C4128A907A803031CD7
:100090004528A807A703031C4928A707A603031C94
:1000A0004D2826308400831307302B052B1384073B
:1000B0002A30040203192B170008F700031D6828D3
:1000C0002B1B68282B1A7028AB19682820306B2846
:1000D000AB152B123030F70777080C1E6D289900EE
:1000E000840A2B1F58288A110A120C2984018313B1
:1000F0001F308305193083169900A6309800903080
:100100008312980083161F149F141F159F11073028
:100110009C00FF308312A00083161F149F141F152C
:100120009F1183121F109412A012200883168700BB
:10013000831220162008831687008312A01120083E
:1001400083168700013083129400003083169400D8
:100150000108C739083881008530831290000030CB
:10016000F800920000308316920007309C000508CA
:100170000330F700F70BBA281C0883120D138316FF
:100180009D0105168312051EC7288316C1288316F4
:1001900005168312051EC728831605168312051E31
:1001A000DD288F018E01831605108312051083163A
:1001B00005168312051AD728CC2883160516831234
:1001C000051AEC28831605108312051483160516EC
:1001D0008312051EE628DD280F08FA000E08F70036
:1001E0000F087A02031DEC287708A1007A08A20004
:1001F000A30123080420A30AF70077080C1EFE2899
:10020000990008302302031DF928003084002208D9
:10021000A5002108A4001B280C30A40024080420F9
:10022000A40AF70077080C1E132999001230240243
:0A023000031D0E298316C128630088
:02400E00F93F78
:00000001FF
